:1018000052C086C06BC06AC069C068C067C066C08D
:1018100065C064C063C062C061C060C05FC05EC0BC
:101820005DC05CC05BC00000EC2DFD2DB7B6B0FC08
:10183000FDCF27BFE895B7B6B0FCFDCF21E1B7B625
:10184000B6FCF4CF0895FFFFFFFFFFFFFFFFFFFF90
:10185000FFFFFFFF090212000101008032090400AE
:1018600000000000000012011001FF000008C01677
:10187000DC050201010200010E0355005300420085
:101880006100730070001C037700770077002E0062
:10189000660069007300630068006C002E0064003D
:1018A00065000403090411241FBECFE5D4E0DEBFA8
:1018B000CDBF10E0A0E6B0E0E8EFFFE102C0059088
:1018C0000D92A836B107D9F710E0A8E6B0E001C044
:1018D0001D92AE39B107E1F72FD18CC391CFA82F5C
:1018E000B92F80E090E041E050EA609530E009C017
:1018F0002D9182279795879510F084279527305E44
:10190000C8F36F5FA8F30895EADF8D939D93089560
:10191000CF93CFB7CF93DF93C395869BE9F7869B91
:101920000BC0869B09C0869B07C0869B05C0869B13
:1019300003C0869B01C089C06F93C0918100DD27E1
:10194000C857DF4F2F9365E5869B03C02F916F919A
:10195000E6CF0F931F934F9320E040E15F9300B3D6
:10196000047406FB27F93F9350E03BE039C0147440
:1019700040642F77012F5F5F1EC0406810B314745E
:101980002F7752501FC0406400B32F770474D1F1F9
:101990005F5F00C023C0406210B32F77147491F1D1
:1019A0005F5F00C025C004741027515012F45D5FC2
:1019B0000000115027952C3F10B3C8F6147401276E
:1019C000015027952C3FC8F64227499300B3047471
:1019D00010274F73115027952C3FA8F64695469532
:1019E00010B3147479F00127015027952C3F98F615
:1019F0006B5A60F3315000B3B0F600C010E41ABF68
:101A0000002717C03B503195C31BD04010E41ABFCC
:101A10000881033CF9F00B34E9F020917F00198133
:101A2000110F1213EDCF093651F10D3211F0013EB5
:101A300039F7009386003F915F914F911F910F916D
:101A40002F916F91CAB7C6FD67CFDF91CF91CFBFFE
:101A5000CF91189520918600222369F3109184007C
:101A6000112339F534303AF130938400209380000B
:101A7000109181003BE0311B309381001CC000912C
:101A800084000130B4F40AE53091610034FD14C0E3
:101A900000936100C4E7D0E013C0052710E000C048
:101AA000000002BB1AC0052710E0221F1DC010E075
:101AB00021C04AE502C032ED432FC4E1D0E032E05C
:101AC00011B31464969A02B311BB54E420E865E3A1
:101AD00020FF052702BB279517951C3FF0F666955A
:101AE000B8F7B1F720FF052702BB279517951C3FD4
:101AF000D0F62795179517FF052700001C3F02BB5E
:101B0000B0F629913A9519F70B7B10918500110FCA
:101B1000C651D04002BB11F010937F0010E41ABFF1
:101B2000006411B31B7B402F4B7B54E05A95F1F7B7
:101B300002BB11BB42BB7FCF11BA80E882BB14BE8F
:101B400081E08BBF82E08BBF879932C288E10FB6FC
:101B5000F89481BD11BC0FBE85B7826085BF8BB77D
:101B600080648BBF8E9A80E006C0EFE9FFE031977A
:101B7000F1F700C000008150C1F78E987894009171
:101B80008400035007FD7AC1209181008CE090E031
:101B9000821B9109EC01C857DF4F209180002D3244
:101BA00009F0E8C0083009F067C123EC2093740005
:101BB0002AE520936100109268004881242F207646
:101BC0003981222309F463C089E690E09093830071
:101BD00080938200333081F59B818C812A81203370
:101BE00039F48370E82FF0E0ED59FF4F808120C079
:101BF000283529F4992371F4E1E0F0E006C020359E
:101C000071F49923A1F4E0E0F0E089E080935700BB
:101C100084910EC0983059F4E3E0F0E0F6CF203A1A
:101C200011F4D3D105C0203C11F46D81D6D180E0F0
:101C300080936C0024E094C0353029F13A3019F1DA
:101C4000832F84508630A8F48A819B8190936E0004
:101C500080936D003930C9F02E8120936F008D8103
:101C60008270809370003093710047FD75C02FEF34
:101C700073C080916000323011F48E7F01C08160AA
:101C80008093600002C021E06BC020E069C02A811F
:101C900010927D00332331F410927E008DE790E0A6
:101CA00022E055C0353019F42093850044C0363009
:101CB000E1F5FC01E657FF4F208185579F4FFC015E
:101CC0008081813019F486E698E104C0823041F4C5
:101CD00084E598E1909383008093820022E121C003
:101CE0008330F1F4222341F482EA98E19093830057
:101CF0008093820024E015C0213041F486E898E109
:101D000090938300809382002CE10BC0223041F439
:101D100088E798E190938300809382002EE001C0D1
:101D200020E080E4809368001BC0383069F03930CF
:101D300029F4209387008DE790E004C08DE790E0C0
:101D40003A3021F020E003C087E890E021E0909352
:101D500083008093820004C080E88093680007C0FD
:101D60008F81882321F48E81821708F4282F2093F5
:101D7000620082C08091680087FF7EC080916F0002
:101D8000801708F4082F801B80936F0011E08111E9
:101D900010E080917100873008F466C07E010FC0AA
:101DA00080916D0090916E009C012F5F3F4F3093AA
:101DB0006E0020936D00F70161917F010ED18E2D91
:101DC0008C1B801768F354C080916D0090916E0059
:101DD00038E18030930708F04DC02E5FF894E09111
:101DE0006D00F0916E008991999131E00C01309372
:101DF0005700E8951124789480916D0090916E00C1
:101E0000029690936E0080936D008F739070009790
:101E100041F0112351F1201740F180917000882387
:101E200021F1F894E0916D00F0916E00329783E01B
:101E300080935700E895789407B600FCFDCFF8949E
:101E4000E0916D00F0916E00329785E0809357002D
:101E5000E895789407B600FCFDCFF89481E1809373
:101E60005700E895789401C020E0201708F4ACCF23
:101E7000112311F010926200109284008091610091
:101E800084FF72C0809162008F3F09F46DC0C82F3B
:101E9000893008F0C8E08C1B809362008091740048
:101EA00098E8892780937400CC2309F44CC0809172
:101EB000680087FF28C080916F008C1708F4C82F36
:101EC0008C1B80936F00D0E005E710E019C0809173
:101ED0007100E0906D00F0906E00873018F0C7013F
:101EE00074D002C0F7018491F80180830F5F1F4F07
:101EF0000894E11CF11CF0926E00E0926D00DF5F2F
:101F0000DC1729F71EC0E0918200F091830086FF64
:101F100009C08C2FA5E7B0E094919D933196815034
:101F2000D9F70BC0DF012C2F85E790E03D91FC0134
:101F30003193CF01FD012150C9F7F0938300E09365
:101F40008200C93058F485E790E06C2FDDDCCC5F6F
:101F5000CC3041F08FEF8093620004C08FEF80930C
:101F60006200CEE1C093610084E190B3947431F4D7
:101F70008150D9F71092850010927F008091600007
:101F8000803130F0879B0FC080916000805109C084
:101F9000879909C080916000823028F080916000AC
:101FA00082508093600080916000882309F0E7CD23
:101FB000F8948E9A12BA1BBE15BE81E08BBF1BBE71
:101FC000E0917200F09173000995E199FECF9FBBFB
:101FD0008EBBE09A99278DB30895262FE199FECF05
:101FE0009FBB8EBB2DBB0FB6F894E29AE19A0FBE51
:081FF00001960895F894FFCF5B
:081FF800FE5AFF1E93070000D2
:0400000300001800E1
:00000001FF
